:103E84000ECF0EBB0EA70E920E7C0E650E4D0E3499
:103E94000E190DFE0DE10DC40DA50D850D640D4229
:103EA4000D1E0CFA0CD40CAE0C860C5D0C330C08F5
:103EB4000BDC0BB00B820B540B250AF50AC40A93D6
:103EC4000A610A2F09FD09CA09960963092F08FC2A
:103ED40008C808950861082E07FB07C807960764F9
:103EE4000733070206D206A206730645061705EA3B
:103EF40005BF059305690540051704F004C904A32B
:103F0400047E045A0437041503F403D303B403965C
:103F14000378035B033F0324030A02F002D702BFC2
:103F240002A80292027C02670253023F022C021A88
:103F3400020801F701E601D601C701B801A9019CF5
:103F4400018E018101740168015D01510146013C4A
:103F540001320128011F0115010D010400FC00F4C8
:103F640000EC00E500DE00D700D000CA00C300BDAD
:103F740000B800B200AD00A700A2009E0099009412
:103F84000090008C008700840080007C007800751D
:103F94000072006E006B0068006500620060005DE6
:103FA400005A0058005500530051004E004C004A7E
:103FB40000480046004400430041003F003E003CEE
:103FC400003A003900370036003500330032003142
:103FD400002F002E002D002C002B002A0029002881
:103FE4000027002600250024002300010C01010401
:103FF40002011E030A960401320502020600640748
:10400400010108000009015A0E01010F000112000C
:104014006413010114013C1501FA1664FA17FFFF39
:104024001D00072000072400022701012F013C3056
:10403400030332010335FFFF3603073CFFFF3DFF57
:10404400FF180002191E461A00021B00022D32C876
:104054002E0001FAFAFA18000019FFFF1A00001BDB
:1040640000002D32C82E0001FAFAFA18000019FFD8
:10407400FF1A00001B00002DFFFF2EFFFFFAFAFAC3
:10004800900786E0FEA3E0FF7457BE0010D39F40E0
:100058000C903FEE12001EE493F599804C9000142A
:10006800E0D394044014900786E0FEA3E0FF903F9D
:10007800EE12001EE493F599802F900014E0D394BB
:10008800034014900786E0FEA3E0FF9040031200AF
:100098001EE493F5998012900786E0FEA3E0FF9096
:1000A800401812001EE493F59990078612000E90EE
:1000B8000786E0FEA3E0FF746C6F4E7003751300B3
:1000C80022900072E0B402087401900072F0D20E1F
:1000D80090013AE090002AF090013BE090002BF06C
:1000E80090013CE090002CF0A20AB3401690013A2F
:1000F800E0700C90013BE0700690013CE0600280EB
:1001080002C20A90013AE0B4300F90013BE0B447D4
:100118000890013CE0643B60028004D20B8002C27C
:100128000BE558B40102800302024B900057E0F53A
:1001380066900062E0F568900063E0F569900074ED
:10014800E0F56A90007AE0900029F090007CE0F5F4
:100158006590007DE0F567900080E0F5649000818F
:10016800E0F563900090E0900041F0900091E090FD
:100178000042F0900092E0900043F0900093E090ED
:100188000044F0900094E0900045F0900095E090D5
:100198000046F0900096E0900047F0900097E090BD
:1001A8000048F0900099E0900033F090009AE090B9
:1001B8000034F090009BE0900035F090009CE090B7
:1001C8000036F0900079E0B4011790000A740FF03F
:1001D800A374FFF090000CE4F0A3F074029000798F
:1001E800F0900079E0B4035990000CE0FEA3E0FF22
:1001F80090000AE0FCA3E0FD12000374101241E431
:1002080074081241D6EF900026F0EF700674FF9044
:100218000026F07400900079F090000BE090002721
:10022800F090000AE0900028F0900026E0900789FE
:10023800F0900027E090078AF0900028E090078B64
:10024800F0803F900081E07006755801756300A248
:100258000AB3402E90013AE090002AF090013BE06A
:1002680090002BF090013CE090002CF090002AE0E8
:10027800700C90002BE0700690002CE06002800269
:10028800C20AE5667003756602E568700375680260
:100298007E837FC2E5668E048F05FF1241C68C39C6
:1002A8008D3AE56975F0FAA4FFAEF0E5688E048F23
:1002B80005FF1241C68C3D8D3E90004FE0F56090E1
:1002C800004DE0FE900069E0B5061890004CE0FE95
:1002D800900068E0B5060C90004BE0FE900059E0F5
:1002E8006E606F900069E07006900068E0600674C8
:1002F80000900059F0900069E0B402089000497439
:1003080001F08005900049E4F0900068E0B402082C
:1003180090004A7401F0800590004AE4F09000686B
:10032800E0600690004AE060028005756003800383
:10033800756004E559B55802D20E900068E0900047
:100348004CF0900069E090004DF0900059E090006A
:100358004BF0740190009EF0740190009FF07400BF
:100368009000A0F074009000A1F074009000A2F03A
:1003780074009000A3F074009000A4F07401900041
:10038800A5F074019000A6F074009000A7F0740026
:100398009000A8F074009000A9F074009000AAF0F2
:1003A80074009000ABF074019000ACF07401900000
:1003B800ADF074009000AEF074009000AFF07400DF
:1003C8009000B0F074009000B1F074009000B2F0AA
:1003D8007401900362F07401900363F07400900359
:1003E80064F07400900365F07400900366F0740084
:1003F800900367F07400900368F074009003A2F013
:1004080074019003A3F074009003A4F074009003A7
:10041800A5F074009003A6F074009003A7F0740090
:100428009003A8F074009003E2F074009003E3F0E6
:1004380074009003E4F074009003E5F074009003F6
:10044800E6F074009003E7F074009003E8F074009D
:10045800900422F07400900423F07401900424F0B6
:100468007400900425F07400900426F07400900441
:1004780027F07400900428F022E5B554F7F5B5E5A7
:10048800B554FDF5B5C2A2C2A1C296C295C2927575
:100498006F00757000C207E5B554FBF5B5755104DA
:1004A800E55104F55290004FE0F560900025E4F026
:1004B800C209E5B554FEF5B5C28E758D00758B0081
:1004C800754C00752600752500D28E22750A0075B8
:1004D8000900AE09AF0A7457BE00039F5003020516
:1004E80091903FEE12001EE49390004E1241FC0FD3
:1004F800BF00010EE0FC903FEE12001EECFEE493FC
:10050800FFEEC39F5026AE09AF0A0FBF00010E9041
:100518003FEE12001EAE09AF0AE493FC903FEE12C4
:10052800001EE49390004E1241FCECF0AE09AF0AB5
:10053800903FEE12001EE49390004E1241FCE0FC46
:10054800903FF012001EECFCE493FDECD39D4019A3
:10055800903FF012001EE493FC903FEE12001EE460
:100568009390004E1241FCECF0AE09AF0A74022FD2
:10057800FF50010E8E098F0A780A740126F650047E
:1005880018E436F640030204DA22750A00750900F9
:10059800AE09AF0A7415BE00039F500302065F90B0
:1005A800404512001EE49390004E1241FC0FBF001C
:1005B800010EE0FC90404512001EECFEE493FFEEB5
:1005C800C39F5026AE09AF0A0FBF00010E904045E9
:1005D80012001EAE09AF0AE493FC90404512001EBB
:1005E800E49390004E1241FCECF0AE09AF0A904043
:1005F8004512001EE49390004E1241FCE0FC90402E
:100608004712001EECFCE493FDECD39D401990408A
:100618004712001EE493FC90404512001EE493909C
:10062800004E1241FCECF0AE09AF0A740F6F4E7029
:1006380006750A15750900AE09AF0A74022FFF5036
:10064800010E8E098F0A780A740126F6500418E400
:1006580036F6400302059822750A00750900AE09AE
:10066800AF0A7415BE00039F500302072D90405A2D
:1006780012001EE49390004E1241FC0FBF00010EC1
:10068800E0FC90405A12001EECFEE493FFEEC39F7C
:100698005026AE09AF0A0FBF00010E90405A120053
:1006A8001EAE09AF0AE493FC90405A12001EE49370
:1006B80090004E1241FCECF0AE09AF0A90405A127D
:1006C800001EE49390004E1241FCE0FC90405C1246
:1006D800001EECFCE493FDECD39D401990405C12A5
:1006E800001EE493FC90405A12001EE49390004EC2
:1006F8001241FCECF0AE09AF0A740F6F4E7006752C
:100708000A15750900AE09AF0A74022FFF50010ED1
:100718008E098F0A780A740126F6500418E436F612
:10072800400302066622750A00750900AE09AF0A81
:100738007415BE00039F50030207FB90406F120020
:100748001EE49390004E1241FC0FBF00010EE0FC26
:1007580090406F12001EECFEE493FFEEC39F5026FC
:10076800AE09AF0A0FBF00010E90406F12001EAE17
:1007780009AF0AE493FC90406F12001EE4939000C6
:100788004E1241FCECF0AE09AF0A90406F12001E09
:10079800E49390004E1241FCE0FC90407112001E60
:1007A800ECFCE493FDECD39D401990407112001EBF
:1007B800E493FC90406F12001EE49390004E1241A7
:1007C800FCECF0AE09AF0A740F6F4E7006750A158F
:1007D800750900AE09AF0A74022FFF50010E8E0989
:1007E8008F0A780A740126F6500418E436F6400396
:1007F80002073422054D22054C22054EC2CF229015
:10080800F800E4936406600280FE75840175A70011
:1008180075FF80900788E4F075C91075A70F75A15A
:10082800C775A70075D90075CEFF75A70F75F1FEBE
:1008380075F2FF75F33775F47875A4BA75A5FF7569
:10084800A60775AE0075AFFF75D48175D5FF75D64F
:10085800FF75D7FFC296C295C2A0C297E5B554BF2F
:10086800F5B5E5B554DFF5B5E5B554EFF5B5E5B53E
:10087800547FF5B5E5B554F7F5B5E5B554FDF5B5CF
:1008880075A70075A20175A14775F80975BC0175B2
:10089800BE0475BD6C75BE0775BDA075BE0875BD77
:1008A8000175BC0075BB1875BC2075BA0875E88061
:1008B80075D11375A70F75E10575E20075C7407509
:1008C8009700759780740A1241B67597C0E59754DA
:1008D80020700280F8758F0275A700D2AF75980056
:1008E80075A90C75A70F75AB4375ADFB75AC1E7577
:1008F800A700758911758E00758C00758A00D2A9BC
:10090800D28C758D00758B00D2ABD28E75CD0075EB
:10091800CC0075CA0075CB00D2ADC2CFD2CA7591D2
:10092800047592007593CD75EF0675D94075CF01A2
:10093800900786E4F0A3F0751300751400C299D2ED
:100948000AC20F12048174C8F5187517001227B36C
:1009580075A70FE5FB90001AF0E5FA90001BF0E58B
:10096800F990001CF075A70090F800E493F50812C0
:1009780028EA122E24900789E0900026F090078A32
:10098800E0900027F090078BE0900028F090078C0B
:10099800E0900029F090078DE0F56690078EE0F56D
:1009A8006890078FE0F569900790E0F56A900791E5
:1009B800E0F565900792E0F567900793E0F564909D
:1009C8000794E0F563900795E090002AF090079669
:1009D800E090002BF0900797E090002CF09007989B
:1009E800E0900041F0900799E0900042F090079A5B
:1009F800E0900043F090079BE0900044F090079C43
:100A0800E0900045F090079DE0900046F090079E2A
:100A1800E0900047F090079FE0900048F09007A012
:100A2800E0900033F09007A1E0900034F09007A226
:100A3800E0900035F09007A3E0900036F074009045
:100A48000082F090013AE0700C90013BE070069053
:100A5800013CE060028004C20A8002D20A90F807D2
:100A6800E493900021F0900021E0440A900021F0E6
:100A7800900021E054FE900021F07406900012F0DE
:100A88007402900013F090F802E493900014F0744C
:100A980003900015F07403900016F0742890001766
:100AA800F07405900018F0900014E0B40406740483
:100AB800900018F0900014E0B40306740390001836
:100AC800F07405900019F090F804E49390001DF07C
:100AD800740090001EF090F805E49390001FF090C9
:100AE800F806E493900020F074FF900022F074540C
:100AF800900125F0746F900126F07479900127F029
:100B0800746F900128F07474900129F07461900159
:100B18002AF0742090012BF0745290012CF074414B
:100B280090012DF0745690012EF0743490012FF03E
:100B38007420900130F07434900131F074539001B6
:100B480032F07450900133F090007AE0D394014071
:100B580006740090007AF075580175590174039075
:100B6800004CF01200C91204D4900014E0B404053B
:100B78001206608011900014E0D394044005120519
:100B880092800312072E1227DFE5B554FEF5B590C3
:100B98000025E4F0900786E4F0A3F075240075239F
:100BA80000754800752A00752900754900753200DE
:100BB800753100754A00755400755500755A0075F1
:100BC800510475520175343C7533007572007571A6
:100BD800007573CD75560075570075430075440050
:100BE800754500754600755B0075470075420075D0
:100BF8004100900006E4F0A3F0900008E4F0A3F0B0
:100C0800755E00755F0090000E74FDF0A374E8F047
:100C1800900023E4F07464900024F0C200D201C272
:100C280002D203754D00756D00C294C293C287C28B
:100C380090C291C20E7E017F00900028E01241E42C
:100C4800900027E02FFF50010E90000AEEF0A3EF6E
:100C5800F0900026E0700674FF900026F090000ADD
:100C6800E0FEA3E0FFEFD394FFEE940F400790005F
:100C78000AE4F0A3F07400900071F0740090007919
:100C8800F07400900082F0740090008DF074009071
:100C980000B4F0E5677003756704743A90074EF086
:100CA80074FD90074FF09003D4E0900414F0D2B094
:100CB800D2B7D2A7D2A6D2B1D2A3C207A2B6B39254
:100CC80004A2B3B39205D29CD2EC75CF01A298B31B
:100CD8004005C298123188E5136006A299B3B34063
:100CE800028005C2991236F8E51464016005E5141E
:100CF800B4040280D5E54DD39405400CE55AC3945D
:100D0800C85002055A754D00E573C394F0501A781F
:100D18007112003FAE71AF72EFD394E8EE940340C6
:100D2800080573757200757100C28E7E047F00E538
:100D38004C1241E4E58D75F004A4FDACF0EF2DFDF7
:100D4800EE3CFCE58B75F04084FF7E00ED2FFFEC58
:100D58003EFE8E258F26D28EA2B6300401B35003F4
:100D6800020EA5A2B6300401B35003020EA5A2B626
:100D780040670554A20F400575FFA0D20FE5B544A2
:100D880001F5B5900024E4F0E554D3956640487C1D
:100D9800837DC2AE25AF261240848E238F24E5487A
:100DA8002FFF50010E74011241D68E238F24852403
:100DB80048755401C28E758D00758B00754C00D234
:100DC8008E7403BE00039F50069000257401F0E561
:100DD80043B40603754300D204A2B6B35003020E0F
:100DE800A5C20490006BE06018123839A200B34025
:100DF80008E5B54408F5B58006E5B554F7F5B580BE
:100E080002C20090006EE0601812398EA202B34050
:100E180008E5B54402F5B58006E5B554FDF5B5809D
:100E280006E5B554FDF5B5A207B34004D2878002A4
:100E3800C287900059E06004D2908002C29090006E
:100E48004AE0B40104D2948002C294900049E0B40C
:100E58000104D2938002C293A209B34004D29180C4
:100E680002C291900018E0FE900014E0C39E400971
:100E7800900014E0D39408400974FB900023F0120A
:100E8800048190001DE0601590001DE0FE900017A1
:100E9800E06E600974FE900023F0120481C2CA7EDD
:100EA800017F00E54E1241E4E5CD2FFF50010E8E83
:100EB800278F28D2CAE565B4014890000EE0FCA34C
:100EC800E0FDEFC39DEE9C4039B208E52A45296054
:100ED80013A208B34008E5B54404F5B58006E5B5A6
:100EE80054FBF5B590000EE0FEA3E0FF900010E083
:100EF800FCA3E0FDEF2DFDEE3CFC90000EECF0A312
:100F0800EDF0A2B3300501B35003020FF3A2B330E2
:100F18000501B35003020FF3A2B35003020FEC050F
:100F280055A20F400575FFA0D20FE5B54401F5B5F0
:100F3800900024E4F0E555D395685003020FEA7C4D
:100F4800EA7D60AE27AF281240848E298F2AE56992
:100F58001241E474FF8E048F05FF1241C68C298D5F
:100F68002AE5492DFD50010C74018C068D071241AC
:100F7800D68E298F2A852A49A209B340157464128E
:100F880041E4900067E08E048F05FF1241C68C296A
:100F98008D2A75550190000EE0FEA3E0FFAC27AD49
:100FA8002812000390000EEEF0A3EFF0E567FF12A1
:100FB80041C6740AFF1241C690007BE08C068D077B
:100FC8001241E474148E048F05FF1241C69000107C
:100FD800ECF0A3EDF0C2CA75CD0075CC00754E00DB
:100FE800D2CAD205A2B3B34002C205900025E0B42C
:100FF8000107E556C394064003021607E56D9027DE
:1010080092F8282873900059E0C394024003021113
:1010180061E551D394015003021161E55175F04027
:10102800A4FFAEF090031212001EE0C395455018BD
:10103800E55175F040A4FFAEF090031112001EE0D8
:10104800F52E752D00021161E55175F040A4FFAE33
:10105800F090031012001EE0C3954540030210FDF6
:10106800E55175F040A4FFAEF090031112001EE5A3
:101078005175F040A4FFAEF0E0FC90030F12001E83
:10108800ECFEE0FFEEC39FFEE5518E0475F040A430
:10109800FFAEF090031012001EE0F40425458C000A
:1010A80088F0A4FFAEF0E5518F048E0575F040A4DA
:1010B800FFAEF090031212001EE55175F040A4FF38
:1010C800AEF0E0FA90031012001EEAFEE0FFEEC355
:1010D8009FFECDCCCD8E071241C6E55175F040A4D8
:1010E800FFAEF090030F12001EE02DFD50010C8C96
:1010F8002D8D2E8064E55175F040A4FFAEF090036D
:101108000F12001EE55175F040A4FFAEF0E0FC9010
:10111800030E12001EECFEE0FFEEC39F8545F0A40F
:10112800FFAEF0E5518F048E0575F040A4FFAEF0D8
:1011380090031012001EE0FECDCCCD8E071241C6E2
:10114800E55175F040A4FFAEF090030E12001EE0CA
:101158002DFD50010C8C2D8D2E756D0102160790FA
:101168000059E0C39402400302131590004FE0D3E6
:10117800955150030212BDE55175F040A4FFAEF041
:1011880090031812001EE0C395455018E55175F0FC
:1011980040A4FFAEF090031712001EE0F52C752B4B
:1011A800000212BDE55175F040A4FFAEF0900316A1
:1011B80012001EE0C395454003021259E55175F02F
:1011C80040A4FFAEF090031712001EE55175F040E1
:1011D800A4FFAEF0E0FC90031512001EECFEE0FF49
:1011E800EEC39FFEE5518E0475F040A4FFAEF0906B
:1011F800031612001EE0F40425458C0088F0A4FFB5
:10120800AEF0E5518F048E0575F040A4FFAEF09066
:10121800031812001EE55175F040A4FFAEF0E0FA85
:1012280090031612001EEAFEE0FFEEC39FFECDCC2F
:10123800CD8E071241C6E55175F040A4FFAEF0907F
:10124800031512001EE02DFD50010C8C2B8D2C80F7
:1012580064E55175F040A4FFAEF090031512001E2E
:10126800E55175F040A4FFAEF0E0FC9003141200C5
:101278001EECFEE0FFEEC39F8545F0A4FFAEF0E54F
:10128800518F048E0575F040A4FFAEF0900316123E
:10129800001EE0FECDCCCD8E071241C6E55175F09B
:1012A80040A4FFAEF090031412001EE02DFD500183
:1012B8000C8C2B8D2CE551B40123E560D3940140AF
:1012C8001CE55604D395514014E545C39405500DCB
:1012D80090035FE0A829B80006952A4002800375AC
:1012E8005102E551B5602290004FE0D39551401965
:1012F800E55175F040A4FFAEF090031712001EE010
:10130800A823B800069524400280020560756D0286
:10131800021607900059E0B4022AE55175F040A47E
:10132800FFAEF090031712001EE0F52C752B00E5B8
:101338005175F040A4FFAEF090030E12001EE0F5C8
:101348002E752D00900059E0B4030F900051E0F580
:101358002C752B00752E00752D00756D0302160770
:10136800E55175F040A4FFAEF090032012001EE096
:10137800C3955A400302143D900049E07036E55188
:10138800D394014029AE23AF24AC2DAD2EEDD39FCD
:10139800EC9E401AE55175F040A4FFAEF090031E94
:1013A80012001EE0A829B80005D3952A5002800231
:1013B80015518034E551D394024029AE23AF24ACB3
:1013C8002DAD2EEDD39FEC9E401AE55175F040A44B
:1013D800FFAEF090031E12001EE0A829B80005D346
:1013E800952A500280021551E551B55237E551C38F
:1013F80095605030E55604D395514028AE23AF246C
:10140800AC2BAD2CEFD39DEE9C4019E55175F04007
:10141800A4FFAEF090031F12001EE0A829B8000632
:10142800952A400280020551C292E5516552600535
:10143800C207755A00756D04021607E55175F0402C
:10144800A4FFAEF090031A12001EE0B40117E55194
:1014580075F040A4FFAEF090032012001EE0240AAD
:10146800C3955A4003021513753064752F00A207FF
:10147800B3500B900060E02405C395454003021566
:1014880013E55175F040A4FFAEF090031D12001E45
:10149800E0C395454064E55175F040A4FFAEF09077
:1014A800031C12001EE55175F040A4FFAEF0E0FCED
:1014B80090031B12001EECFEE0FFEEC39F8545F073
:1014C800A4FFAEF0E5518F048E0575F040A4FFAE81
:1014D800F090031D12001EE0FECDCCCD8E07124108
:1014E800C6E55175F040A4FFAEF090031B12001E34
:1014F800E02DFD50010C8C2F8D30AE23AF24AC2F86
:10150800AD30EFD39DEE9C4002D207756D050216F3
:1015180007E551B40109900059E0C3940240030261
:1015280015E7900358E0D3954550030215E790035B
:1015380056E0C395455040900357E0FE900355E0B0
:10154800F4042EFE900356E0F40425458E0088F03E
:10155800A4FFAEF0900358E0FC900356E0F4042C8E
:101568008E048F05FF1241C6900355E02DFD5001F2
:101578000C8C2B8D2C802C900355E0FE900354E0AE
:10158800F4042E8545F0A4FFAEF0900356E08E04D7
:101598008F05FF1241C6900354E02DFD50010C8CBD
:1015A8002B8D2CE551C395605030E55604D39551E9
:1015B8004028AE23AF24AC2BAD2CEFD39DEE9C403E
:1015C80019E55175F040A4FFAEF090031F12001EFC
:1015D800E0A829B80006952A4002800375510290B8
:1015E8000049E0B40106E5516401600280037551C9
:0F15F80002E55165526005C207755A00756D0016
:1027920002100D02116702131B0213680214430296
:0227A200151907
:10160700900050E02402A823B80007D39524400295
:10161700C207900025E0B40109900059E0C3940384
:10162700400302178F900049E060030216DEE55180
:10163700D394014034E55175F040A4FFAEF0900318
:101647001412001EE0A823B8001FD39524401AE502
:101657005175F040A4FFAEF090031F12001EE0A8E2
:1016670029B80005D3952A500280021551E551D3B8
:101677009401402FE55175F040A4FFAEF09003129E
:1016870012001EE0C39545501AE55175F040A4FFBE
:10169700AEF090031E12001EE0A829B80005D395EE
:1016A7002A500280021551E551D394014022E55694
:1016B70004C39551501AE55175F040A4FFAEF09060
:1016C700031E12001EE0A829B80005D3952A500270
:1016D70080021551021784E551D394024034E55135
:1016E70075F040A4FFAEF090031412001EE0A8238B
:1016F700B8001FD39524401AE55175F040A4FFAEFA
:10170700F090031F12001EE0A829B80005D3952A00
:10171700500280021551E551D39402402FE55175CF
:10172700F040A4FFAEF090031212001EE0C39545EF
:10173700501AE55175F040A4FFAEF090031E120059
:101747001EE0A829B80005D3952A5002800215513A
:10175700E551D394024022E55604C39551501AE54A
:101767005175F040A4FFAEF090031E12001EE0A8D2
:1017770029B80005D3952A500280021551E5516515
:10178700526005C207755A00900060E0D395455036
:1017970009900054E0C395455002C207900059E0F4
:1017A70070030219F4A2A5B34008A2A4B340030230
:1017B70019DDAE35AF367441D39F749C9E400578D2
:1017C7003512003FAE35AF36EFB48806EEB41302DC
:1017D70080030219BAA2A5500302187D900059E0B0
:1017E700B4010B90004FE0D3956040020560900074
:1017F70059E0B40254E55175F040A4FFAEF09003F0
:101807002012001EE0C3955A503F90004FE0D39539
:10181700514021E55604D395514019E55175F040E3
:10182700A4FFAEF090031412001EE0A823B8000630
:10183700952440028002055190004FE0F560E55184
:1018470065526005C207755A00900059E0B4032637
:1018570090004FE0D395514008E55604D395515079
:10186700028002055190004FE0F560E55165526036
:1018770005C207755A00A2A450030219BA9000596D
:10188700E0B4016E900049E07035E551D394014012
:1018970029E55175F040A4FFAEF090031E12001E1B
:1018A700E0A829B8000FD3952A400A1551755A00A8
:1018B700855160800385516080037560018033E541
:1018C70051D394024029E55175F040A4FFAEF09042
:1018D700031E12001EE0A829B8000FD3952A400A5C
:1018E7001551755A008551608003855160800375D5
:1018F7006002900059E0D3940150030219AEE551FC
:1019070075F040A4FFAEF090032012001EE0C395CF
:101917005A40030219AE900049E07041E551D39453
:10192700014034E55175F040A4FFAEF09003111269
:10193700001EE0A823B8001FD39524401AE551756F
:10194700F040A4FFAEF090031E12001EE0A829B8D5
:101957000005D3952A500280021551803FE551D3E7
:1019670094024034E55175F040A4FFAEF0900311A6
:1019770012001EE0A823B8001FD39524401AE55192
:1019870075F040A4FFAEF090031E12001EE0A829D8
:10199700B80005D3952A500280021551E5516552CA
:1019A7006005C207755A00E556B40704055E800353
:1019B700755E00E563B4010EAE35AF36EF64407077
:1019C70005EE649C6002800EA2A54003755801A233
:1019D700A44003755802A2A5B3B35006A2A4B3B39B
:1019E70040028006753600753500021AE2A2A5B3DB
:1019F7004008A2A4B34003021ACEAE35AF367441F5
:101A0700D39F749C9E4005783512003FAE35AF36A4
:101A1700EFB48806EEB413028003021ACEA2A540E3
:101A27006F900068E0605A90004AE0B401079000A8
:101A37004AE4F0800690004A7401F090004AE07092
:101A470005756003800375600490004AE0B40104E3
:101A5700D2948002C294E551B4041AE55175F0405E
:101A6700A4FFAEF090031E12001EE0A829B80005DF
:101A7700D3952A50028008755103C207755A008012
:101A870003756004E556B40704055E8003755E00C0
:101A9700A2A44033900069E06021900049E0B401BE
:101AA70007900049E4F080069000497401F0900027
:101AB70049E0B40104D2938002C293E556B4070407
:101AC700055E8003755E00A2A5B3B35006A2A4B35A
:101AD700B340028006753600753500E558655960D4
:101AE70006900082E06003021C6AC29C75140075B0
:101AF7001300C2CAE5589027A4F828287380121249
:101B07002E24800D122EFD8008122FD6800312304E
:011B1700AF1E
:0F27A400021B04021B06021B0B021B10021B155B
:101B1800900029E090007AF0E566900057F0E568BB
:101B2800900062F0E569900063F0E56A900074F057
:101B3800E56590007CF0E56790007DF0E564900035
:101B480080F0E563900081F090002AE090013AF07F
:101B580090002BE090013BF090002CE090013CF0CD
:101B6800900041E0900090F0900042E0900091F0E9
:101B7800900043E0900092F0900044E0900093F0D1
:101B8800900045E0900094F0900046E0900095F0B9
:101B9800900047E0900096F0900048E0900097F0A1
:101BA800900033E0900099F0900034E090009AF0B3
:101BB800900035E090009BF0900036E090009CF09B
:101BC8007400900082F07454900125F0746F9001B5
:101BD80026F07479900127F0746F900128F07474DE
:101BE800900129F0746190012AF0742090012BF083
:101BF800745290012CF0744190012DF074569001AC
:101C08002EF0743490012FF07420900130F0743469
:101C1800900131F07453900132F07450900133F018
:101C28009003D4E0900414F0743A90074EF074FDD9
:101C380090074FF01200C9900004E4F0A3F0900060
:101C4800067475F0A37430F09000087475F0A374EE
:101C580030F0855859D2CA754C00D29C741B90003C
:101C680023F0E556C394065005E551B55202806746
:101C7800C207E55175F040A4FFAEF09003221200B0
:101C88001EE030E003D38001C3920CE55175F040AB
:101C9800A4FFAEF090032312001EE030E003D380CF
:101CA80001C3920DE55175F040A4FFAEF0900324F6
:101CB80012001EE030E003D38001C392A085515288
:101CC800AE29AF2A7405BE00039F5007E545D3949B
:101CD8000550028002D292E556D394055003021DA6
:101CE800E9C207E551D394014073E55175F040A46A
:101CF800FFAEF090031E12001EE0A829B80007D31B
:101D0800952A40021551E5516552604EE55175F02E
:101D180040A4FFAEF090032212001EE030E003D38F
:101D28008001C3920CE55175F040A4FFAEF090031A
:101D38002312001EE030E003D38001C3920DE55169
:101D480075F040A4FFAEF090032412001EE030E0CE
:101D580003D38001C392A0855152021DE9E556B410
:101D680006279000ACE030E003D38001C3920C90CA
:101D780000ADE030E003D38001C3920D9000AEE0E7
:101D880030E003D38001C392A0E556B40727900042
:101D9800A5E030E003D38001C3920C9000A6E030A8
:101DA800E003D38001C3920D9000A7E030E003D395
:101DB8008001C392A0E556B4082790009EE030E069
:101DC80003D38001C3920C90009FE030E003D380DE
:101DD80001C3920D9000A0E030E003D38001C392CC
:101DE800A0900072E06058E54575F00284FF7E001F
:101DF80090014E12001EE0F55CE54775F00A84FF7D
:101E08007E0090024E12001EE0F55DE55C255DD374
:101E18009464400BE55C255DC39464F55C800375B0
:101E28005C00E55C75F00284FF7E008F5CEFC39474
:101E3800335007EF24CDF55C8003755CFF801CE50B
:101E48004575F00284FF7E0090014E12001EE07579
:101E5800F00284FF7E00EF24CDF55CE595C3955C28
:101E68004004C2A28002D2A2A207B34005E556B43C
:101E780007037573CDE595C395734004C2A180022D
:101E8800D2A1E54575F00284FF7E00900180120022
:101E98001EE075F00284FF7E00EF24CDF56FE59516
:101EA800C3956F5006A20CB3B340028004D296804B
:101EB80002C296E54575F00284FF7E009001B212D9
:101EC800001EE075F00284FF7E00EF24CDF570E57A
:101ED80095C395705006A20DB3B340028004D29505
:101EE8008002C295E543C3940640030224EFA2EDA5
:101EF800B350030224EFC2EDE54360030220517E94
:101F0800017F00E5BE1241E4E5BD2FFF50010E90B0
:101F18000000EEF0A3EFF0900029E0B401177E0F67
:101F28007FFF900000E0FCA3E0FD1200039000009A
:101F3800EEF0A3EFF0900079E0B4025B900000E0CF
:101F4800FEA3E0FF90000AE0FCA3E0FDEDD39FECC8
:101F58009E400F900000E0F8A3E090000AC8F0A3AC
:101F6800C8F0900000E0FEA3E0FF90000CE0FCA3A6
:101F7800E0FDEFD39DEE9C400F900000E0F8A3E059
:101F880090000CC8F0A3C8F0900000E0FEA3E0FFAA
:101F980074041241D68F44900079E070609000007C
:101FA800E0FEA3E0FF90000AE0FCA3E0FDEFD39D74
:101FB800EE9C400D120003900000EEF0A3EFF080BD
:101FC80007900000E4F0A3F0900000E0FEA3E0FF1B
:101FD80074101241E4900026E08E048F05FF124130
:101FE800C6900000ECF0A3EDF07400D39D74019C42
:101FF8004008900001E0F54480037544FFE544750E
:10200800F00AA4FFAEF074198E048F05FF1241C6C2
:102018008D45ED2532FFAE3150010E74011241D6C7
:102028008F45854532753100EFD39462400375457D
:1020380062900072E064016006900066E0600280D1
:1020480005754301800375BB17E543B4010280039E
:102058000221417E017F00E5BE1241E4E5BD2FFF6C
:1020680050010E900000EEF0A3EFF0900072E0B483
:10207800017EE53445336025AC33AD341DBDFF0129
:102088001C8F028E038C068D07903E8412002EE46E
:1020980093FE740193FFEFC39AEE9B40028005788C
:1020A8003312420EAE33AF3474B3BE0025D39F4013
:1020B80021900000E0FCA3E0FD0FBF00010E903E60
:1020C8008412002EE493FE740193FFEDC39FEC9EEF
:1020D80040028005783312003FAE33AF34E56A1210
:1020E80041E474648E048F05FF1241C68D47803326
:1020F800900066E0602D900000E0FEA3E0FFEFD3C3
:102108009400EE9408400F900066E0B40104C20900
:102118008002D209800D900066E0B40104D20980E3
:1021280002C209900072E064026006900066E060F6
:102138000575BB168003754302E543B402028003AC
:1021480002222F7E017F00E5BE1241E4E5BD2FFF8C
:1021580050010E900000EEF0A3EFF0900072E0B492
:10216800027EE53445336025AC33AD341DBDFF0137
:102178001C8F028E038C068D07903D1A12002EE4E8
:1021880093FE740193FFEFC39AEE9B40028005789B
:102198003312420EAE33AF3474B3BE0025D39F4022
:1021A80021900000E0FCA3E0FD0FBF00010E903D70
:1021B8001A12002EE493FE740193FFEDC39FEC9E68
:1021C80040028005783312003FAE33AF34E56A121F
:1021D80041E474648E048F05FF1241C68D47803335
:1021E800900066E0602D900000E0FEA3E0FFEFD3D2
:1021F8009400EE9408400F900066E0B40104C20910
:102208008002D209800D900066E0B40104D20980F2
:1022180002C209900072E07003754700900066E002
:102228007002C20975BB1FE543B403457E017F00F8
:10223800E5BE1241E4E5BD2FFF50010E900000EE0F
:10224800F0A3EFF074091241E474E68E048F05FFE1
:102258001241C68C418D42E54A2DFD50010C740196
:102268008C068D071241D68E418F4285424A75BB36
:1022780019E543B4040280030223D77E017F00E5F9
:10228800BE1241E4E5BD2FFF50010E900000EEF0B4
:10229800A3EFF074041241D68F4BE564B4010280B9
:1022A80003022364756B00756B00E56BD3940740DC
:1022B80003022351E56B9000411241FCE0D3954B9A
:1022C800501AE56B9000411241FCE0F404254BFEE6
:1022D800E56B9000371241FCEEF08017E56B90003B
:1022E800411241FCE0C3954BFEE56B90003712416B
:1022F800FCEEF0E56BC394044009900084E0C395BC
:102308006B503BE56B6029E56B9000371241FCFE92
:10231800E0FFEE90003FE0D39F4013E56B9000375D
:102328001241FCE090003FF0E56B900040F0800E19
:10233800900037E090003FF07400900040F0786B18
:10234800740126F640030222B2900040E0F404240F
:1023580008F556E556D394054002C292E564D39435
:1023680001402FE54BD3946E4004D2108002C21076
:10237800755605E564B40205A210B34002800375E2
:102388005607E564B40306A210B3B3400280037590
:102398005607E55765566008E55104F552855657C6
:1023A800E556B40708E5B54480F5B58006E5B554AB
:1023B8007FF5B5E55664066005E556B40808E5B549
:1023C8004410F5B58006E5B554EFF5B575BB13E5D2
:1023D80043B4050280030224EB7E017F00E5BE12B0
:1023E80041E4E5BD2FFF50010E900000EEF0A3EF91
:1023F800F074041241D68F46E563B40202800302EA
:1024080024E8756B00756B00E56BD39403400302F9
:10241800249FE56B9000331241FCE0D39546501A97
:10242800E56B9000331241FCE0F4042546FEE56BB1
:1024380090002D1241FCEEF08017E56B90003312EE
:1024480041FCE0C39546FEE56B90002D1241FCEE81
:10245800F0E56B6029E56B90002D1241FCFEE0FF72
:10246800EE900031E0D39F4013E56B90002D1241B0
:10247800FCE0900031F0E56B900032F0800E9000A7
:102488002DE0900031F07400900032F0786B740108
:1024980026F64003022410900082E07043E52A45A6
:1024A800296036E558C39403500A900032E004C30B
:1024B800940340028007900032E004F558E558D3B1
:1024C8009402400A900032E004D39402500280073C
:1024D800900032E004F5588007900032E004F55887
:1024E80075BB180543D2ECE55ED39404500302266D
:1024F8005275CF01C2A2AE35AF367488D39F74131C
:102508009E4005A2A5B34014AE35AF367488D39F5C
:1025180074139E4005A2A4B3400280487835120087
:102528003FAE35AF36EFB4883BEEB41337A2A5B350
:10253800500990004FE0D395515002800405518016
:1025480011A2A5B3500890004FE0655160028002C7
:10255800D207A2A4B35007E551D3940150028004D6
:102568001551C207A2A5B3B35006A2A4B3B3400243
:102578008006753600753500E5516552604EE551A7
:1025880075F040A4FFAEF090032212001EE030E088
:1025980003D38001C3920CE55175F040A4FFAEF05F
:1025A80090032312001EE030E003D38001C3920D94
:1025B800E55175F040A4FFAEF090032412001EE030
:1025C80030E003D38001C392A0855152A207400591
:1025D8007573CD80037573FFE595C395734004C289
:1025E800A18002D2A1E54575F00284FF7E0090012A
:1025F8008012001EE075F00284FF7E00EF24CDF506
:102608006FE595C3956F5006A20CB3B340028004E2
:10261800D2968002C296E54575F00284FF7E00904E
:1026280001B212001EE075F00284FF7E00EF24CD97
:10263800F570E595C395705006A20DB3B3400280BE
:1026480004D2958002C2950224F9A20FB3500DAEB0
:1026580025AF2674E8C39F74039E4002800575FF6A
:10266800A0D20FAE25AF26EFD39420EE944E5003A0
:10267800022766120481C28E758D00758B00754C19
:1026880000D28EC2077572007571007573CD7551D1
:1026980004752400752300755400755A00C287908C
:1026A8000059E06004D2908002C29090004AE0B4E1
:1026B8000104D2948002C294900049E0B40104D28B
:1026C800938002C293A209B34004D2918002C291BE
:1026D80090006BE06018123839A200B34008E5B5E5
:1026E8004408F5B58006E5B554F7F5B58002C20093
:1026F80090006EE0601812398EA202B34008E5B56A
:102708004402F5B58006E5B554FDF5B58006E5B596
:1027180054FDF5B590000E74FDF0A374E8F0E543A0
:10272800B40603754300900025E4F075260075256E
:1027380000758D00758B00754C00900024E0C394E3
:10274800035008900024E004F080067403900024ED
:10275800F0900024E0B40306E5B554FEF5B5AE27C5
:10276800AF28EFD39410EE9427401CC2CA75CD0051
:1027780075CC00752800752700D2CA754E00752AD9
:0A27880000752900755500020CD2FF
:103B40000000010001320164019601960200021298
:103B500002240200020003000340038003C00400AB
:103B60000440048004C005000600060006000600AC
:103B7000060006000600060000FF01310163019502
:103B800001FF01FF0211022302FF02FF02FF033FB8
:103B9000037F03BF03FF043F047F04BF04FF05FF4F
:103BA00006FF06FF06FF06FF06FF06FF06FF06FFED
:103BB0000FAA0FA50F9F0F9A0F940F8D0F870F80DD
:103BC0000F780F710F680F600F570F4E0F450F3BA7
:103BD0000F300F250F1A0F0E0F020EF50EE80EDB39
:103BE0000ECC0EBE0EAE0E9F0E8E0E7D0E6C0E5ABD
:103BF0000E470E340E200E0C0DF70DE20DCB0DB559
:103C00000D9D0D850D6D0D540D3A0D200D050CE922
:103C10000CCE0CB10C940C760C580C3A0C1B0BFB14
:103C20000BDB0BBB0B9A0B790B570B350B130AF104
:103C30000ACE0AAB0A870A640A400A1C09F809D4AA
:103C400009B0098C09670943091F08FB08D608B2A7
:103C5000088E086A0846082307FF07DC07B907969D
:103C600007730751072F070D06EC06CA06AA068937
:103C700006690649062A060A05EC05CD05B0059237
:103C800005750558053C0520050504EA04CF04B573
:103C9000049C04820469045104390422040B03F4D3
:103CA00003DE03C803B2039D038903750361034D5B
:103CB000033B03280316030402F202E102D102C00F
:103CC00002B002A002910282027302650257024909
:103CD000023C022F02220216020901FD01F201E656
:103CE00001DB01D001C601BB01B101A7019D019417
:103CF000018B018201790170016801600158015056
:103D00000148014101390132012B0125011E011831
:103D10000111010B010500FF00FA0FA60FA00F997A
:103D20000F920F8B0F840F7C0F740F6B0F620F5865
:103D30000F4E0F430F380F2C0F1F0F120F050EF7EA
:103D40000EE80ED80EC80EB70EA50E930E800E6CA0
:103D50000E580E420E2C0E150DFD0DE40DCB0DB1BF
:103D60000D950D790D5D0D3F0D200D010CE10CC081
:103D70000C9E0C7C0C590C350C100BEA0BC40B9EE2
:103D80000B760B4F0B260AFD0AD40AAA0A800A55A5
:103D90000A2A09FF09D409A8097C0950092508F94C
:103DA00008CD08A10875084A081E07F307C8079D33
:103DB00007730749072006F706CE06A6067E0657B4
:103DC0000630060A05E405BF059B05770554053254
:103DD000051004EF04CE04AE048F047104530435BF
:103DE000041903FD03E203C703AD0394037B0363DC
:103DF000034B0334031E030802F302DE02CA02B6B9
:103E000002A30291027F026D025C024C023C022C72
:103E1000021D020E020001F201E401D701CA01BE37
:103E200001B101A6019A018F0185017A0170016635
:103E3000015D0153014A014101390131012901218B
:103E400001190112010B010400FD00F700F000EA66
:103E500000E400DE00D900D300CE00C900C400BFDA
:103E600000BA00B500B100AD00A800A400A0009CFD
:103E7000009900950091008E008A008700840081DF
:043E8000007E007B45
:1027B300751A00751900AE19AF1AAC17AD18EDC331
:1027C3009FEC9E401674FF1241B675CF01781A74C0
:1027D3000126F6500418E436F650DB22900786E40F
:1027E300F0A3F0751000750F00751300751400C287
:1027F30011D21222C2AF75D900758F0375B7A575B3
:10280300B7F190F800E4F0758F0175B7A575B7F1CE
:10281300E50890F800F075B7A575B7F190F801E4F5
:10282300F075B7A575B7F190079DE090F802F075C4
:10283300B7A575B7F19007A1E090F803F075B7A5B8
:1028430075B7F190079EE090F804F075B7A575B7DA
:10285300F190079FE090F805F075B7A575B7F19073
:1028630007A0E090F806F075B7A575B7F19007A239
:10287300E090F807F0758F0075D940D2AF2290072A
:1028830088E0B4AB61C2AF75D90075B62275F52285
:10289300758F0375B7A575B7F1740090F600F075E1
:1028A3008F01750A00750900AE09AF0A7413BE00E3
:1028B300279F402475B7A575B7F190078912001EAD
:1028C300E0FC90F60012001EECF0780A740126F684
:1028D300500418E436F650D0758F0075F51175B6AF
:1028E3002075D940D2AF22C2AF75D90075F52275D4
:1028F3000A00750900AE09AF0A7413BE00229F4097
:102903001F90F60012001EE493FC90078912001E2C
:10291300ECF0780A740126F6500418E436F650D524
:1029230075F51175D940D2AF22900788E0B4AA0299
:102933008003022A69C2AF75D90075B62275F522E4
:10294300758F0375B7A575B7F1740090EE00F07538
:10295300B7A575B7F1740090F000F075B7A575B71A
:10296300F1740090F200F075B7A575B7F17400909B
:10297300F400F0758F01750A00750900AE09AF0AFE
:1029830074FFC39F74019E402475B7A575B7F1907A
:10299300004E12001EE0FC90EE0012001EECF078D8
:1029A3000A740126F6500418E436F650CF750A006F
:1029B300750900AE09AF0A74FFC39F74019E4024DA
:1029C30075B7A575B7F190024E12001EE0FC90F0AA
:1029D3000012001EECF0780A740126F6500418E485
:1029E30036F650CF750A00750900AE09AF0A74FFB9
:1029F300C39F74019E402475B7A575B7F190044E2B
:102A030012001EE0FC90F20012001EECF0780A7433
:102A13000126F6500418E436F650CF750A007509FE
:102A230000AE09AF0A74FFC39F74019E402475B7BB
:102A3300A575B7F190064E12001EE0FC90F400124B
:102A4300001EECF0780A740126F6500418E436F6FA
:102A530050CF758F0075F51175B62075D940D2AF7B
:102A6300743A90074EF022900788E0B4AA028003DC
:102A7300022BA7C2AF75D90075B62275F522758FE3
:102A83000375B7A575B7F1740090E600F075B7A5A7
:102A930075B7F1740090E800F075B7A575B7F174D8
:102AA3000090EA00F075B7A575B7F1740090EC00DB
:102AB300F0758F01750A00750900AE09AF0A74FF3E
:102AC300C39F74019E402475B7A575B7F190004E5E
:102AD30012001EE0FC90E60012001EECF0780A746F
:102AE3000126F6500418E436F650CF750A0075092E
:102AF30000AE09AF0A74FFC39F74019E402475B7EB
:102B0300A575B7F190024E12001EE0FC90E800128A
:102B1300001EECF0780A740126F6500418E436F629
:102B230050CF750A00750900AE09AF0A74FFC39F41
:102B330074019E402475B7A575B7F190044E120039
:102B43001EE0FC90EA0012001EECF0780A740126E5
:102B5300F6500418E436F650CF750A00750900AE36
:102B630009AF0A74FFC39F74019E402475B7A5750E
:102B7300B7F190064E12001EE0FC90EC0012001E0E
:102B8300ECF0780A740126F6500418E436F650CFB8
:102B9300758F0075F51175B62075D940D2AF743AAB
:102BA30090074EF022900788E0B4AA028003022C1B
:102BB300E5C2AF75D90075B62275F522758F037519
:102BC300B7A575B7F1740090DE00F075B7A575B7BA
:102BD300F1740090E000F075B7A575B7F17400903B
:102BE300E200F075B7A575B7F1740090E400F075D5
:102BF3008F01750A00750900AE09AF0A74FFC39F00
:102C030074019E402475B7A575B7F190004E12006C
:102C13001EE0FC90DE0012001EECF0780A74012620
:102C2300F6500418E436F650CF750A00750900AE65
:102C330009AF0A74FFC39F74019E402475B7A5753D
:102C4300B7F190024E12001EE0FC90E00012001E4D
:102C5300ECF0780A740126F6500418E436F650CFE7
:102C6300750A00750900AE09AF0A74FFC39F7401AA
:102C73009E402475B7A575B7F190044E12001EE06F
:102C8300FC90E20012001EECF0780A740126F65064
:102C93000418E436F650CF750A00750900AE09AF83
:102CA3000A74FFC39F74019E402475B7A575B7F1DD
:102CB30090064E12001EE0FC90E40012001EECF0A1
:102CC300780A740126F6500418E436F650CF758F4F
:102CD3000075F51175B62075D940D2AF743A9007D7
:102CE3004EF022900788E0B4AA028003022E23C28A
:102CF300AF75D90075B62275F522758F0375B7A523
:102D030075B7F1740090D600F075B7A575B7F17477
:102D13000090D800F075B7A575B7F1740090DA008C
:102D2300F075B7A575B7F1740090DC00F0758F01ED
:102D3300750A00750900AE09AF0A74FFC39F7401D9
:102D43009E402475B7A575B7F190004E12001EE0A2
:102D5300FC90D60012001EECF0780A740126F6509F
:102D63000418E436F650CF750A00750900AE09AFB2
:102D73000A74FFC39F74019E402475B7A575B7F10C
:102D830090024E12001EE0FC90D80012001EECF0E0
:102D9300780A740126F6500418E436F650CF750A03
:102DA30000750900AE09AF0A74FFC39F74019E400A
:102DB3002475B7A575B7F190044E12001EE0FC9080
:102DC300DA0012001EECF0780A740126F65004189B
:102DD300E436F650CF750A00750900AE09AF0A74E0
:102DE300FFC39F74019E402475B7A575B7F1900684
:102DF3004E12001EE0FC90DC0012001EECF0780A7C
:102E0300740126F6500418E436F650CF758F00751A
:102E1300F51175B62075D940D2AF743A90074EF0CC
:102E230022C2AF75D90075F522750A00750900AE87
:102E330009AF0A74FFC39F74019E401F90EE0012F6
:102E4300001EE493FC90004E12001EECF0780A740E
:102E53000126F6500418E436F650D4750A007509B5
:102E630000AE09AF0A74FFC39F74019E401F90F028
:102E73000012001EE493FC90024E12001EECF07848
:102E83000A740126F6500418E436F650D4750A0085
:102E9300750900AE09AF0A74FFC39F74019E401FFA
:102EA30090F20012001EE493FC90044E12001EECFC
:102EB300F0780A740126F6500418E436F650D475F7
:102EC3000A00750900AE09AF0A74FFC39F74019E1F
:102ED300401F90F40012001EE493FC90064E120073
:102EE3001EECF0780A740126F6500418E436F65006
:102EF300D475F51175D940D2AF22C2AF75D900751B
:102F0300F522750A00750900AE09AF0A74FFC39F65
:102F130074019E401F90E60012001EE493FC900093
:102F23004E12001EECF0780A740126F6500418E4E1
:102F330036F650D4750A00750900AE09AF0A74FF5E
:102F4300C39F74019E401F90E80012001EE493FC8F
:102F530090024E12001EECF0780A740126F650041B
:102F630018E436F650D4750A00750900AE09AF0AA5
:102F730074FFC39F74019E401F90EA0012001EE479
:102F830093FC90044E12001EECF0780A740126F6AE
:102F9300500418E436F650D4750A00750900AE09DA
:102FA300AF0A74FFC39F74019E401F90EC00120090
:102FB3001EE493FC90064E12001EECF0780A740196
:102FC30026F6500418E436F650D475F51175D94039
:102FD300D2AF22C2AF75D90075F522750A00750903
:102FE30000AE09AF0A74FFC39F74019E401F90DEB9
:102FF3000012001EE493FC90004E12001EECF078C9
:103003000A740126F6500418E436F650D4750A0003
:10301300750900AE09AF0A74FFC39F74019E401F78
:1030230090E00012001EE493FC90024E12001EEC8E
:10303300F0780A740126F6500418E436F650D47575
:103043000A00750900AE09AF0A74FFC39F74019E9D
:10305300401F90E20012001EE493FC90044E120005
:103063001EECF0780A740126F6500418E436F65084
:10307300D4750A00750900AE09AF0A74FFC39F74C3
:10308300019E401F90E40012001EE493FC90064E44
:1030930012001EECF0780A740126F6500418E43688
:1030A300F650D475F51175D940D2AF22C2AF75D998
:1030B3000075F522750A00750900AE09AF0A74FFA1
:1030C300C39F74019E401F90D60012001EE493FC20
:1030D30090004E12001EECF0780A740126F650049C
:1030E30018E436F650D4750A00750900AE09AF0A24
:1030F30074FFC39F74019E401F90D80012001EE40A
:1031030093FC90024E12001EECF0780A740126F62E
:10311300500418E436F650D4750A00750900AE0958
:10312300AF0A74FFC39F74019E401F90DA00120020
:103133001EE493FC90044E12001EECF0780A740116
:1031430026F6500418E436F650D4750A00750900C3
:10315300AE09AF0A74FFC39F74019E401F90DC0049
:1031630012001EE493FC90064E12001EECF0780A47
:10317300740126F6500418E436F650D475F511752B
:10318300D940D2AF22E51464046006E59964FF6078
:10319300028031A2114004D2118027E51460087423
:1031A300E62514900023F0E513600874F0251390CE
:1031B3000023F0E514B4010280FE751400751300BA
:1031C300C2118002C211E514903AE3F828287375FE
:1031D3001400E599B4FF03751301E599B4FE037573
:1031E3001302E599B4FD03751303E599B4FC037564
:1031F3001304E599B4FA03751305E599B4FB067551
:103203001401120481E599B4F906751404120481BA
:10321300E599D394E54007E599C394F040028016FD
:103223008599157514027E017F00E515C394E61296
:1032330041E48E0D8F0E900786E4F0A3F0E599D359
:1032430094C44007E599C394E64002802885991504
:1032530075140374E5C39515F50E750D00AE0DAF2A
:103263000E903B4012002EE493F87401939007866E
:10327300C8F0A3C8F0D2990236F7900786E0FEA300
:10328300E0FFEFC39400EE94054009EFD394FFEE03
:1032930094064013900786E0FEA3E0FF90004E12D1
:1032A300001EE599F0800385996C90078612000E45
:1032B300900786E0FEA3E0FFEFB40106EEB4070239
:1032C300800302350790074EE0B43C0280030235C9
:1032D30007A20AB35005A20BB340030233FAC29C00
:1032E30090007AE090078CF0900057E090078DF003
:1032F300900062E090078EF0900063E090078FF0FB
:10330300900074E0900790F090007CE0900791F0BB
:1033130090007DE0900792F0900080E0900793F09A
:10332300900081E0900794F090013AE0900795F0C7
:1033330090013BE0900796F090013CE0900797F0F6
:10334300900090E0900798F0900091E0900799F03A
:10335300900092E090079AF0900093E090079BF022
:10336300900094E090079CF0900095E090079DF00A
:10337300900096E090079EF0900097E090079FF0F2
:10338300900099E09007A0F090009AE09007A1F0D8
:1033930090009BE09007A2F090009CE09007A3F0C0
:1033A3007400900082F01200C974AB900788F01289
:0A33B300288174AA900788F0E558FD
:063AE3000231D202327D27
:1033BD00903B04F8282873801212292C800D122AB4
:0B33CD006A8008122BA88003122CE677
:0F3B04000233C40233C60233CB0233D00233D5AF
:1033D800900788E4F090013AE0700C90013BE070AF
:1033E8000690013CE060028004C20A8002D20A0210
:1033F80034FCC29C900078E0900789F090005EE071
:1034080090078AF090005FE090078BF090007AE0D8
:1034180090078CF0900057E090078DF0900062E0E4
:1034280090078EF0900063E090078FF0900074E0B2
:10343800900790F090007CE0900791F090007DE07C
:10344800900792F0900080E0900793F0900081E060
:10345800900794F090013AE0900795F090013BE0D6
:10346800900796F090013CE0900797F0900090E06C
:10347800900798F0900091E0900799F0900092E002
:1034880090079AF0900093E090079BF0900094E0EA
:1034980090079CF0900095E090079DF0900096E0D2
:1034A80090079EF0900097E090079FF0900099E0B9
:1034B8009007A0F090009AE09007A1F090009BE0A0
:1034C8009007A2F090009CE09007A3F07400900091
:1034D80082F074AB900788F012288174AA9007884C
:1034E800F012292C122A6A122BA8122CE6D29C75EB
:1034F80099FB80FED29C7514007513007599FB0228
:1035080036F7900786E0FEA3E0FFEF4E7006859938
:1035180010750F00900786E0FEA3E0FF74016F4E60
:10352800701BAC0FAD10AA0DAB0EED2BFBEC3AFAED
:103538008A068B0790004E12001EE599F0900786C8
:1035480012000E900786E0FEA3E0FF74026F4E7033
:103558000C1200C98515997514007513000236F709
:10356800900786E0FEA3E0FF90004E12001EE5994A
:10357800F090078612000E900786E0FEA3E0FFACED
:103588000DAD0E8F028E038C068D07903B781200CE
:103598002EE493F9740193FEEAD39EEB99400985D2
:1035A80015997514007513000236F7900786E0FE2A
:1035B800A3E0FF90004E12001EE599F090078612D6
:1035C800000E900786E0FEA3E0FFEFB40006EEB41D
:1035D800010280030236F790001CE0D394C7400B29
:1035E80090001CE0C394C8F516801A90001CE0D324
:1035F8009463400B90001CE0C39464F51680069019
:10360800001CE0F516E51675F002A4FFAEF08F6B0E
:10361800EF90004E1241FCEFFCE0FDEC90005112DF
:1036280041FCEDFCE0FDEC2DB5160280030236E905
:103638000FEF90004E1241FCE56BFFE0FCEF9000AD
:10364800521241FCECFFE0FCEFC39CB5160280036C
:103658000236E9E56B9000501241FCE56BFFE0FC97
:10366800EF9000531241FCECFFE0FCEF2CB5167113
:10367800E56B9000541241FCE0C3951690079DF04D
:10368800E56B9000551241FCE0C3951690079EF03B
:10369800E56B9000581241FCE0C3951690079FF027
:1036A800E56B9000591241FCE0C395169007A0F015
:1036B800E56B90005A1241FCE0C395169007A1F003
:1036C800E56B90005B1241FCE0C395169007A2F0F1
:1036D8001227F77599F97518647517001227B380C2
:0F36E800FE7599FF7518647517001227B380FEE1
:093AE90002350A0235680235B30A
:1036F70022E513903AF2F8282873023838900786A3
:10370700E0FEA3E0FF90001212001EE0F59990077B
:103717008612000E900786E0FEA3E0FF74116F4E3D
:10372700700375130002383885629902383890079C
:1037370086E0FEA3E0FF90004E12001EE0F599EF31
:10374700B40107EEB4070375130090078612000E45
:07375700023838900787E0FB
:0F3AF20002370102370402372F02373502375AE5
:10375E00903B13F828287385249902382D852A99D1
:10376E0002382D85449902382D85479902382D85CA
:10377E00519902382D85609902382D855699023857
:10378E002D85589902382D756E00900069E07006EF
:10379E00900068E060028016A2A44006E56E440424
:1037AE00F56EA2A54006E56E4402F56E801A9000F5
:1037BE004AE0B40106E56E4410F56E900049E0B49F
:1037CE000106E56E4420F56EA207B34006E56E4491
:1037DE0001F56EA209B34006E56E4408F56E856EDE
:1037EE0099803CA212B340077599FAC2128017A2B3
:1037FE000EB3400575990F800B900023E0F599905C
:10380E000023E4F0C20E80178542998012854B99F1
:0F381E00800D85469980087599FC80037513000D
:103B130002376502376B02377102377702377D024E
:103B2300378302378902378F0237950237F102381C
:0D3B33001602381B02382002382502382AFD
:0B382D0090078612000E800312004876
:033B010002383552
:103838002290006BE0B4010385241190006BE0B482
:103848000203852A1190006BE0B4030385441190AC
:10385800006BE0B4040385471190006BE0B40503E6
:1038680085511190006BE0B4060385561190006BEA
:10387800E0B4070385581190006CE0FE90006DE0FD
:10388800C39E500302390F90006BE0D39404402C80
:1038980090006CE0D39511500990006DE0C395112C
:1038A80050028002D20090006CE0D395115009902C
:1038B800006DE0C395115002C200804990006BE092
:1038C800B4041890006DE0C395115002D200900026
:1038D8006CE0D395114002C200802A90006CE0C3CE
:1038E8009511500990006DE0D3951150028002D2D5
:1038F8000090006CE0D39511500990006DE0C395DD
:10390800115002C200807E90006BE0D39404402CDA
:1039180090006CE0C39511400990006DE0D39511BB
:1039280040028002C20090006CE0C39511400990EB
:10393800006DE0D395114002D200804990006BE001
:10394800B4041890006CE0C395115002C2009000B6
:103958006DE0D395114002D200802A90006CE0C33C
:103968009511400990006DE0D395114002D2009066
:10397800006CE0D39511400990006DE0C3951140AB
:10398800028002C2002290006EE0B4010385241177
:1039980090006EE0B40203852A1190006EE0B40333
:1039A8000385441190006EE0B4040385471190002C
:1039B8006EE0B4050385511190006EE0B4060385EE
:1039C800561190006EE0B4070385581190006FE01F
:1039D800FE900070E0C39E5003023A6490006EE0CF
:1039E800D39404402C90006FE0D3951150099000B7
:1039F80070E0C3951150028002D20290006FE0D3AC
:103A080095115009900070E0C395115002C20280D0
:103A18004990006EE0B40418900070E0C39511500E
:103A280002D20290006FE0D395114002C202802AB0
:103A380090006FE0C395115009900070E0D3951184
:103A480050028002D20290006FE0D3951150099085
:103A58000070E0C395115002C202807E90006EE0B3
:103A6800D39404402C90006FE0C395114009900056
:103A780070E0D3951140028002C20290006FE0C34B
:103A880095114009900070E0D395114002D2028050
:103A98004990006EE0B4041890006FE0C39511508F
:103AA80002C202900070E0D395114002D202802A2F
:103AB80090006FE0C395114009900070E0D3951114
:103AC8004002D20290006FE0D39511400990007037
:0B3AD800E0C3951140028002C20222F0
:0941FC002582F5825002058322A0
:10002E00EF2F500205832582F582E5833E2EF58360
:01003E00229F
:08000300C3EF9DFFEE9CFE22FD
:08003F000806B60002180622B3
:0D000E00A3E004F070061241F2E004F022BD
:08420E000816B6FF0218162283
:0E41D600048007C3CE13CECF13CFD5E0F62260
:10408400BC000FBE0008ED8FF084FFADF022E4FE0B
:10409400FF22BE000DEF60FE54F0606F20E70302C4
:1040A400413AEAC0E0EBC0E078017A0075F001EE35
:1040B40020E710EF25E0FFEE33FE0AC5F023C5F03C
:1040C40030E7F0EA5407F9096A7A007B00600108D6
:1040D400C3EC9E40167004ED9F4010ED9FFDEC9ED6
:1040E400FCE5F0CA4ACA03F5F08005E5F003F5F0F3
:1040F400C3EE13FEEF13FFD9D77908CACBCAD8D0C1
:10410400EAFEEBFFD0E0FBD0E0FA22EC8FF084FC77
:10411400ED54F045F0C48FF084FEEDC454F045F046
:10412400C48FF084FDEEC4FE54F02DFFEE540F3C1A
:10413400FEADF07C0022790078008FF0EC7E082040
:10414400E70DC3CD33CD33C933C9C833C8DEF084DA
:1041540049F9E5F08FF0BE00E6FD7C00E9FFE8FEDA
:014164002238
:0E41E400F88FF0A4FFE5F0CE88F0A42EFE22A6
:1041B600600D782B0241C0007830D8FED5E0F82299
:1041C600EEC0E07E00124084EFFDEEFCD0E0FE2261
:03000B000241654A
:03001B000241801F
:03002B0002419BF4
:03000000024205B4
:0942050075817475D000020807F0
:0B001E00E5822FF582E5833EF583228A
:0A41F2000582D58202158315822292
:10416500C0E0C0F0C083C082C0D075D0001207FC8B
:10417500D0D0D082D083D0F0D0E032C0E0C0F0C043
:1041850083C082C0D075D0001207FFD0D0D082D0B6
:1041950083D0F0D0E032C0E0C0F0C083C082C0D090
:1041A50075D000120802D0D0D082D083D0F0D0E0F4
:0141B50032D7
:00000001FF
